:020000040000FA
:103388004F6C6420426F6F746D616E616765720087
:102D8E002804E00DE00FBE88CA009037F2F400B4BC
:102D9E004841FD04E118E48002000D03E108E480DF
:102DAE000200E6F880F9E009CA00FC36E00BE00A02
:102DBE00E008E6F92000CA00DE2BE028CA001E2C2F
:102DCE00CA009037CA00C437CA00FE3706F488130B
:102DDE00B840CA00FE37F0E406FEF401E6FB80F9C7
:102DEE00E00CF4800200C08AE019E008CA00162048
:102DFE00E009E008CA00042FBF88E6F98873E6F8F8
:102E0E0002B4F01999882D03498D2DFC28112989BA
:102E1E00D08448403D04E118F7F8D7B50D02F78E7F
:102E2E00D7B5F3F8D7B53D0D0D02CA009037E01AAD
:102E3E00E009E018CA00B02149803DF70D09CA002B
:102E4E009037E00AE009E008CA00B02149803DF75A
:102E5E00E6869EC4E018CA00B82BE6F81200CA0037
:102E6E00C02A0E00CA009037CA00641349803D0D77
:102E7E00CA00FE3706F48813B840A8D0E008CA008E
:102E8E00C02AE6F81200CA00C02A9A001700F04EB7
:102E9E00204D284146F400808D11F04F49802D05BC
:102EAE00E018CA00C02AE00F0D04E028CA00C02AAC
:102EBE00E01FCA00FE37F0E406FEF401CA00FE373A
:102ECE00F0D4A840204D284146F400808DCBD71079
:102EDE004000F2F40450F2F5065026F4800038500B
:102EEE003D04E018CA00AC270DBDCA00FE3706F43B
:062EFE00F401B8400DB71D
:10010000D180E612C000D1A0E60AF00EE60BE00EA8
:10011000E60CD00ED1A0E68AAF04E68BAF04E68CE5
:10012000AF040A86FF8A1A86C4D61A8901FF0A8993
:100130006F06D1A0E6EE0300E6E80000E6EA45001F
:10014000E60C0510E68ABFC4E60D0020E68B4DC61E
:10015000E60A0CFAE60900FCE6000000E6010000F1
:10016000E6020300F2F4AEFFF6F400B4E60800FC89
:10017000B54AB5B5E6F000B4E6F90000E6F89C0033
:10018000F01870192D2FA758A7A7E005DC099828AB
:100190002D29F032DC099848AAF21DE0AAF20EF0EF
:1001A000F0347C330EF306F300FDE0154C5491500F
:1001B000685BB853084128213DF30DE5DC09983808
:1001C000A758A7A7DC44B9A30831184076F300C0AC
:1001D00028217DF60DD8A758A7A7B9A40841282142
:1001E0007DFA0DD1E6F90000E6F87E39A758A7A7F9
:1001F000E6030300DC09A8282D3E08821890AAF225
:100200002BF0F04266F2FF3F3D05E004DC09A82830
:1002100008821890DC09A838088218908AF406E051
:10022000F6F306FEDC09A83808821890DC09A9A8B4
:1002300008811890B9A308318AF406E08AF304E033
:100240000603010076F300C0A758A7A728213DEEBA
:100250009AF8CC0008810DCAC0435C1376F300FD08
:10026000E014F1A54C458AF203709140684B0D01F2
:0A027000784BB8430DBBFA008E2D49
:1027AC00ECFDF0D8D120BE88CC00CC00CA009A3702
:1027BC00CA00F837CA009037F3F8D7B549813D0BFA
:1027CC00E006E00708611870F046F05726F4001098
:1027DC0038508DF80D09E006E00708611870F046D6
:1027EC00F057284038518DF9CA009037F04D2981A7
:1027FC002D1829828D1F2D3109833D41E6FC800067
:10280C00E6F4BA29CA004A38F0A4F0B5E6F880F923
:10281C00E009CA005C39E6F480F9E005DA004438D6
:10282C000D2ED7104000F2F41050F2F51250DA00D1
:10283C0044380D25E6FC8000E6F4C429CA004A3869
:10284C00F0A4F0B5E6F880F9E009CA005C39E6F4CA
:10285C0080F9E005DA0044380D12E6FC8000E6F45D
:10286C00CE29CA004A38F0A4F0B5E6F880F9E009A0
:10287C00CA005C39E6F480F9E005DA004438FCFD66
:02288C00CB007F
:08288E00E6F48000E005CB0038
:06289600E034E005CB0078
:08289C00E6F40002E005CB00A8
:0628A400E004E005CB009A
:0C28AA00F2F47CF066F4FF00E005CB00C7
:1028B6002804F04809803D0CE118B980E138E4802D
:1028C6000100E118E4800200E108E48003000D0B3A
:1028D600E108B980E7F8FF00E4800100E480020027
:1028E600E108E4800300F04066F4FF3FF2F504FEE1
:0428F600E041CB00F2
:1028FA00ECFDECFEECFF06F0F8FFE00DE004E6F577
:10290A001000F0EDF0F5D7104000F2F40850F2F59F
:10291A000A50B840C4500200D7104000F2F40C50DC
:10292A00F2F50E50C4400400C4500600E6F8120046
:10293A00CA00C02AE6F82100CA00C02AD4700200E0
:10294A00A860F0460842B840DC07A846F08E08E2C4
:10295A00DC0FB84886FDFF1F3D0BE6F81100CA00E0
:10296A00C02AE6F82200CA00C02ACA0090370D0E13
:10297A0046FD00403D0BE6F81200CA00C02AE6F800
:10298A002100CA00C02AE00DCA009037D4400400D2
:10299A00D450060028423850C4400400C4500600EF
:1029AA0070453DCC06F00800FCFFFCFEFCFDCB00A8
:0A29BA00660C0F00FA000000CB00CD
:0A29C400660C0F00FA000000CB00C3
:0A29CE00660C0F00FA000000CB00B9
:100B4C00ECFDECFEECFFF0E8F0F906F0CEFFE084F3
:100B5C00C4401200DC09D4480600C4401000E00D6B
:100B6C00DC09F488010047F8FF003D10E088CA005A
:100B7C00B42FBF88CA009037CA00482F49832DFC78
:100B8C00CA009037CA005237EA004C13DC0FF48EBF
:100B9C0001004983EA304C13E108EA005813EA00DB
:100BAC004C13CA009037D4601200F04E0046C4407B
:100BBC000400C4F00600F04E004DC4400800C4F020
:100BCC000A00D4500600D4400400DC05F484010073
:100BDC00C0840846D45012000045C4401200D450C2
:100BEC000600D4400400DC05F4840100C0850856DE
:100BFC00D44010002045C4401000D4500600D4400E
:100C0C000400DC05A9842982EA20760D2982EA8079
:100C1C00240EEA205E0F2982EA206C102981EA203A
:100C2C0030112983EA20DC112981EA20781207F897
:100C3C000A00EA30EC12D4500600D4400400DC0563
:100C4C00F4840200E4800C00D4500600D44004006C
:100C5C00DC05F4840300E4800D00D4500600D4407D
:100C6C000400DC05F4840400E4800E00D45006007B
:100C7C00D4400400DC05F4840500E4800F00D4505B
:100C8C000600D4400400DC05F4840100C084E005B7
:100C9C008850F0C4D4500800D44006000846F0A494
:100CAC00F0B5D4400E00D450100006F51000F084BE
:100CBC00F095CA00C0380802E11CD4500A00D44098
:100CCC000800DC05B9C4D4500A00D4400800DC0587
:100CDC00E4C40100D4500A00D4400800DC05E4C48C
:100CEC000600D4400C00D4500E00F1C8D4500A00B9
:100CFC00D4400800DC05E4C40200D4400C00D450FD
:100D0C000E00F0657C847C855C867046F1C8D450FE
:100D1C000A00D4400800DC05E4C40300D4500E00E3
:100D2C00F045E005F1C8D4500A00D4400800DC05B9
:100D3C00E4C40400D4400C00D4500E00F0457C8474
:100D4C00E005F1C8D4500A00D4400800DC05E4C426
:100D5C000500D4500A00D4400800DC05F4840100DE
:100D6C00C084084600D4EA004C13D4500600D4408A
:100D7C000400DC05F4840600B980E12CD4500A0090
:100D8C00D4400800DC05B9C4E11CD4500A00D4409E
:100D9C000800DC05E4C40100E10CD4500A00D44086
:100DAC000800DC05E4C40200D4500A00D44008005A
:100DBC00DC05E4C40300D4500A00D4400800DC0570
:100DCC00E4C40400D4500A00D4400800DC05E4C498
:100DDC000500E11CD4500A00D4400800DC05E4C432
:100DEC000600D4500A00D4400800DC05F48401004D
:100DFC00C084084600D4F08DCA00B42FBF88CA0046
:100E0C00482F49832DFCCA009037A980C088CA009E
:100E1C00AC27E108EA005813D4500600D440040073
:100E2C00DC05F4840100C084084600D4D4500600CC
:100E3C00D4400400DC05F4840200E4800C00D4509F
:100E4C000600D4400400DC05F4840300E4800D00AB
:100E5C00D4500600D4400400DC05F4840400E48083
:100E6C000E00D4500600D4400400DC05F4840500C8
:100E7C00E4800F00E13CD4500A00D4400800DC05AB
:100E8C00B9C4D4500600D4400400DC05F48401003D
:100E9C00D4700A00D4600800DC07E4860100D4405A
:100EAC000C00D4500E00F1C8D4500A00D4400800F5
:100EBC00DC05E4C40200D4400C00D4500E00F065F4
:100ECC007C847C855C867046F1C8D4500A00D44082
:100EDC000800DC05E4C40300D4500E00F045E00526
:100EEC00F1C8D4500A00D4400800DC05E4C4040066
:100EFC00D4400C00D4500E00F0457C84E005F1C8C1
:100F0C00D4500A00D4400800DC05E4C40500D450D9
:100F1C000A00D4400800DC05F4840100C084E0051C
:100F2C008850F0C4D4400E00D450100006F51000C8
:100F3C00F0A4F0B5D4500C00D4400A000846F0845C
:100F4C00F095CA00C0380802E004C4401000EA0062
:100F5C004C13E0A4E0058850F0C4E6FA1C33E6FB21
:100F6C000000E6F816000080E00906F8004016F9CB
:100F7C000000CA00C0380802E6F41000E0058850F2
:100F8C00F0C4E6FA2633E6FB0000E6F82400008005
:100F9C00E00906F8004016F90000CA00C038080243
:100FAC00E7F86000E4801E00E118E4801F00E1789F
:100FBC00E4802000E128E4802100E14CD4500A00B8
:100FCC00D4400800DC05B9C4E7FC1E00D4500A006C
:100FDC00D4400800DC05E4C40100E10CD4500A0044
:100FEC00D4400800DC05E4C40200D4500A00D4400C
:100FFC000800DC05E4C40300D4500A00D440080007
:10100C00DC05E4C40400D4500A00D4400800DC051C
:10101C00E4C40500D4500A00D4400800DC05F48474
:10102C000100C084084600D4E6F41E00E005885098
:10103C00F0C4E6FA160000A0E00B06FA004016FB1E
:10104C000000D4500C00D4400A000846F084F095FF
:10105C00CA00C0380802E004C4401000EA004C1377
:10106C00D4500600D4400400DC05F4840100B9809F
:10107C00E16CD4500A00D4400800DC05B9C4A9C006
:10108C00D4500A00D4400800DC05E4C40100E10C93
:10109C00D4500A00D4400800DC05E4C40200D4504B
:1010AC000A00D4400800DC05E4C40300D4500A0054
:1010BC00D4400800DC05E4C40400D4500A00D44039
:1010CC000800DC05E4C40500A980C084084600D4EF
:1010DC00E108E48002000D1CF4800200C086D450AC
:1010EC000600D44004000046DC05F4E40600B1E040
:1010FC00F4800200C086D4500A00D4400800004698
:10110C00DC05E4E40600F48002000981E4800200BE
:10111C00A9A0F4800200418A8DDFE004C4401000D5
:10112C00EA004C13E6F40050E005F6F4DEB5F6F5F3
:10113C00E0B5E17CD4500A00D4400800DC05B9C409
:10114C00E7FC1A00D4500A00D4400800DC05E4C4C3
:10115C000100E10CD4500A00D4400800DC05E4C4C2
:10116C000200D4500A00D4400800DC05E4C403009B
:10117C00D4500A00D4400800DC05E4C40400D45068
:10118C000A00D4400800DC05E4C40500D4500A0071
:10119C00D4400800DC05F4840100C084084600D467
:1011AC00E6F41A00E0058850F0C4F2FBE0B5F2FA60
:1011BC00DEB5D4500C00D4400A000846F084F095FB
:1011CC00CA00C0380802E004C4401000EA004C1306
:1011DC00E1ACD4500A00D4400800DC05B9C4E11CD1
:1011EC00D4500A00D4400800DC05E4C40100E10C32
:1011FC00D4500A00D4400800DC05E4C40200D450EA
:10120C000A00D4400800DC05E4C40300D4500A00F2
:10121C00D4400800DC05E4C40400D4500A00D440D7
:10122C000800DC05E4C4050008D7F2F5E0B5F2F4DB
:10123C00DEB5DC05A84446F4FFFF3D08D4500A0097
:10124C00D4400800DC05E4C406000D08E11CD450B1
:10125C000A00D4400800DC05E4C40600F08DCA0086
:10126C00B42FBF88CA00FA28E1080D700F00E1BC4A
:10127C00D4500A00D4400800DC05B9C4E11CD45099
:10128C000A00D4400800DC05E4C40100E10CD45091
:10129C000A00D4400800DC05E4C40200D4500A0063
:1012AC00D4400800DC05E4C40300D4500A00D44048
:1012BC000800DC05E4C40400D4500A00D440080043
:1012CC00DC05E4C40500E11CD4500A00D44008003D
:1012DC00DC05E4C4060008D7E004C44010000D305F
:1012EC00E7FCFF00D4500A00D4400800DC05B9C468
:1012FC00E10CD4500A00D4400800DC05E4C4010021
:10130C00D4500A00D4400800DC05E4C40200D450D8
:10131C000A00D4400800DC05E4C40300D4500A00E1
:10132C00D4400800DC05E4C40400D4500A00D440C6
:10133C000800DC05E4C4050008D6E004C440100035
:10134C00D44010004840EAE0AE0BF04D06F03200FD
:08135C00FCFFFCFEFCFDCB00D0
:10331C005345524E554D424552005553422D436F25
:10332C006D706163740000000000000207008000F3
:10333C000000000000000040000000000000424DB2
:10334C0020563200000000005553422D436F6D7023
:10335C006163740000000000000106002446572D34
:10336C00494E464F24004F6C6420426F6F746D6160
:0C337C006E6167657200424D2056320001
:10136400ECFDECFEECFF06F0EAFFE148E48004004B
:10137400D120BE88CC00CC00CA006A2FF064F0757E
:10138400C4400600C45008007065EA20F419E1085E
:10139400E48004000E00D4F00800D4E00600DC0F62
:1013A400D44E0600C4401200E084C4401400E00D92
:1013B400F3F8D7B549813D0AF09FF08ECA004C0B73
:1013C400C08DE004C4401200EA00E419DC0FF48E7E
:1013D400010047F8FF003D07E008CA00B42FBF88AA
:1013E400E108EA00FA19D4500800D4400600DC05EC
:1013F400F48401004983EA30E419E008CA00B42FF8
:10140400BF88E108EA00FA19EA00E419CA00903733
:10141400D4701400D4900800D4800600F04800472B
:10142400C4400A00C4900C00008DF0E8F0F9D430F8
:101434000C00D4200A00DC0399A2C0A6F0A608A1DF
:10144400F04A0047C4401400D4401200204AC4406B
:101454001200DC03A98247F80B00EA90BA19C08491
:101464005C2406F46C149C04EA009814EA00FC144E
:10147400EA007415EA00D015EA006C16EA001817A1
:10148400EA00A617EA00CE17EA001A18EA00A01824
:10149400EA00CA18E064E0058850F0C4E6FA823332
:1014A400E6FB0000F04E0843F05FF084F09FCA00B2
:1014B400C0380802E10CDC0FE4CE0D00E12CDC0F97
:1014C400E4CE0E00E17CDC0FE4CE0F00E10CDC1F67
:1014D400E4CE1000E4CE0100DC0FE4CE0200E7FC11
:1014E4001000DC1FB9CEA98EC084084100D4E004EA
:1014F400C4401200EA00E419D4500C00D4400A009D
:10150400DC05A9842982B980E108E48002000D1673
:10151400F4200200C028D4500C00D4400A00004833
:10152400DC05F4E40300B1E0F04E0048DC0FE4E431
:101534000300F48002000981E4800200A9A0F48081
:101544000200418A8DE5E11CDC0FE4CE0100E10CD0
:10155400DC0FE4CE0200A9C009C2DC1FB9CEA98EFB
:10156400C084084100D4E004C4401200EA00E41935
:10157400D4500C00D4400A00DC05F4840300B98084
:10158400E12CDC0FE4CE0100E10CDC0FE4CE020020
:10159400E12CDC1FB9CEA98EC084084100D4F08DA3
:1015A400CA00B42FBF88CA00482F49832DFCCA0043
:1015B4009037E00AE008E009CA004222A980C08806
:1015C400CA00AC27F4800400EA00FA19D4500C00D5
:1015D400D4400A00DC05F4840300E4800E00D450F7
:1015E4000C00D4400A00DC05F4840400E4800F00FD
:1015F400D4500C00D4400A00DC05F4840500E480D7
:101604001000D4500C00D4400A00DC05F484060019
:10161400E4801100D4700C00D4600A00DC07A986B1
:10162400C0842846E0058850F0C40867F0A6F0B7E7
:10163400D4401000D450120006F51000F084F09548
:10164400CA00C0380802E13CDC0FE4CE0100E10C22
:10165400DC0FE4CE0200E12CDC1FB9CEA98EC084DD
:10166400084100D4EA00E419D4500C00D4400A0024
:10167400DC05F4840700B980D4500C00D4400A007F
:10168400DC05F4840300E4800E00D4500C00D44044
:101694000A00DC05F4840400E4800F00D4500C003C
:1016A400D4400A00DC05F4840500E4801000D45022
:1016B4000C00D4400A00DC05F4840600E480110028
:1016C400E14CDC0FE4CE0100E10CDC0FE4CE0200BF
:1016D400A980C084E0058850F0C4D4401000D450E0
:1016E400120006F51000F0A4F0B5F04E0843F05FC8
:1016F400F084F09FCA00C0380802A9C009C2DC1FE8
:10170400B9CEA98EC084084100D4E004C4401200BC
:10171400EA00E419E10CDC0FE4CE0300E11CDC0F69
:04172400E4CE04000B
:10172800E16CDC0FE4CE0500E10CDC0FE4CE060032
:10173800E0A4E0058850F0C4E6FA1C33E6FB00009C
:10174800F04E0847F05FF084F09FCA00C0380802E6
:10175800E6F41000E0058850F0C4E6FA2633E6FB0C
:101768000000F04E06F41100F05FF084F09FCA000C
:10177800C0380802E15CDC0FE4CE0100E10CDC0FAC
:10178800E4CE0200E7FC2000DC1FB9CEA98EC0849D
:10179800084100D4E004C4401200EA00E419E16CF6
:1017A800DC0FE4CE0100E10CDC0FE4CE0200E12CFA
:1017B800DC1FB9CEA98EC084084100D4E004C4401F
:1017C8001200EA00E419E6F41E00E0058850F0C4AF
:1017D800E6FA0050E6FB4000F04E0843F05FF08464
:1017E800F09FCA00C0380802E17CDC0FE4CE01009B
:1017F800E10CDC0FE4CE0200E7FC1E00DC1FB9CED2
:10180800A98EC084084100D4E004C4401200EA0054
:10181800E419E18CDC0FE4CE0100E12CDC1FB9CE29
:10182800A98EC084084100D4D7104000F2F40450B7
:10183800F2F5065026F4FFFF36F5FFFF3D0BDC0FEF
:10184800E4CE0200F08DCA00B42FBF88F4800400F3
:10185800EA00FA19D7104000F2F40C50F2F50E50D5
:101868008850F0C4D7104000F2F40850F2F50A503E
:10187800F0A4F0B5E008E6F91000CA00C038080284
:10188800E10CDC0FE4CE0200F08DCA00B42FBF8853
:10189800F4800400EA00FA190F00E19CDC0FE4CEA2
:1018A8000100E10CDC0FE4CE0200E12CDC1FB9CE14
:1018B800A98EC084084100D4E004C4401200EA00A4
:1018C800E419E016DC1FE4CE0300E4DE0400E026A1
:1018D800DC1FE4CE0500E4DE0600E6F60005E6F7C8
:1018E8000203DC3FE4CE0700E4DE0800E4EE090072
:1018F800E4FE0A00CA00AA28DC3FE48E0B00E49E3E
:101908000C00E4AE0D00E4BE0E00CA008E28F064A0
:10191800DC1FE4CE0F00E4DE1000CA009628F06455
:10192800DC1FE4CE1100E4DE1200CA009C28F0643B
:10193800DC1FE4CE1300E4DE1400CA00A428F0641F
:10194800DC1FE4CE1500E4DE1600E108E4800200A6
:10195800F4800200C088CA00B628F0600061F4C6AE
:101968000200C0C85C28F06E0068F07F06F6170019
:10197800E042CA00AC380001F4800200F1A809A1D5
:10198800E4A0020047FA08008DE3E1ACDC0FE4CEE6
:101998000100E10CDC0FE4CE0200E7FC3600DC1F9E
:1019A800B9CEA98EC084084100D4E004C440120016
:1019B8000D15E118F7F8D7B5E6F97273E6F802B431
:1019C80028810881E9893DFDD4900800D48006006B
:1019D800CA004C0BC08DE004C4401200D440120071
:1019E8004840EAE01014F08DCA00B42FBF88F48094
:0E19F800040006F01600FCFFFCFEFCFDCB0018
:1033A200ECFDECFEF0D8E00E0D0D5EE6E6F8E093E3
:1033B200E049CA0004385FE6E6F8E093E049CA0053
:1033C200043808E1F05DF04E418A8DEFFCFEFCFD11
:0233D200CB002E
:1033D400C6030300EC00C6871000EC06EC07ECF112
:1033E400ECF2ECF3ECF4ECF5ECF6ECF7ECF8ECF9CD
:1033F400ECFAECFBECFC5EE78EE38FE26EE76FE643
:10340400E018BBCDE6F820A1E079CA0004380DF835
:10341400C6030300EC00C6871000EC06EC07ECF1D1
:10342400ECF2ECF3ECF4ECF5ECF6ECF7ECF8ECF98C
:10343400ECFAECFBECFC5EE78EE38FE26EE76FE602
:10344400E028BBADE6F820A1E079CA0004380DF805
:10345400C6030300EC00C6871000EC06EC07ECF191
:10346400ECF2ECF3ECF4ECF5ECF6ECF7ECF8ECF94C
:10347400ECFAECFBECFC5EE78EE38FE26EE76FE6C2
:10348400E038BB8DE6F820A1E079CA0004380DF8D5
:10349400C6030300EC00C6871000EC06EC07ECF151
:1034A400ECF2ECF3ECF4ECF5ECF6ECF7ECF8ECF90C
:1034B400ECFAECFBECFCECFD5EE78EE38FE26EE7EE
:1034C4006FE6F2F4ACFF9AF40200E04D0D13F2F44F
:1034D400ACFF9AF40210E05D0D0DF2F4ACFF9AF427
:1034E4000220E06D0D07F2F4ACFF9AF40230E07DA7
:1034F4000D01E08DF04DC088CA00A233E6F820A18A
:08350400E079CA0004380DF65D
:102BDE008AF81400F6F8E2B5F6F9E4B566C4BF005B
:102BEE00F04AC0855C25F04BC0840045F6F488FFA2
:102BFE00D19066E0FCFF76E002000D02E128CB00EA
:042C0E00E108CB000E
:0C2C120066C4BF007EE6E6C40000CB00F4
:102C1E00F04809802D1129822D130981EA308C2D5F
:102C2E00E018CA00B82B7FE6E6F8F401E009CA0006
:102C3E00043876C44000CB007EE666C4BF00CB00ED
:102C4E00E018CA00B82B7EE6E6F8F401E009CA00E7
:102C5E0004387FE6E7FC8000F2F2E2B5F2F3E4B569
:102C6E00F04206F41F00F0531850DC05B9C4E7FC1F
:102C7E00FF00F08206F81000F0931890DC09B9C836
:102C8E00F0A206FA1100F0B318B0DC0BB9CA06F2C6
:102C9E0012001830DC03B9C2F2F4E2B5F2F5E4B575
:102CAE0006F413001850DC05B9C4F2F4E2B5F2F5DF
:102CBE00E4B506F414001850DC05B9C4F2F4E2B51C
:102CCE00F2F5E4B506F415001850DC05B9C4F2F4BB
:102CDE00E2B5F2F5E4B506F416001850DC05B9C4F9
:102CEE00F2F4E2B5F2F5E4B506F417001850DC057F
:102CFE00B9C4E10CF2F4E2B5F2F5E4B508461850A9
:102D0E00DC05B9C4E7FC1800F2F4E2B5F2F5E4B55F
:102D1E0008471850DC05B9C4E7FC5E00F2F4E2B5D2
:102D2E00F2F5E4B506F408001850DC05B9C4E7FC6A
:102D3E001000F2F4E2B5F2F5E4B508441850DC05E3
:102D4E00B9C4E19CF2F4E2B5F2F5E4B5DC05B9C420
:102D5E00E1AC0D06F2F4E2B5F2F5E4B5DC05B9C46A
:102D6E00F2F8E2B5F2F9E4B5DC09A9A88AF5F200A9
:102D7E0077FA1000DC09B9A8E008CA00B82BCB001E
:06397E000140D4B5F00089
:063984000140D5B5F00082
:06398A000140D6B500006B
:1029D800E018BB6BE048BB70E018CA00B82BE018E1
:0429E800EA001E2CB7
:1029EC00C2F4D6B59AF40200E018BB5DC2F4D6B5B9
:1029FC007C249AF40200E048BB5DC2F4D6B57C346A
:0C2A0C009AF40300E018CA00B82BCB00BD
:102A1800ECFEECFFF0E8F0F98AE00410E11875F834
:102A2800D6B50D04E7F8FE0065F8D6B58AE204309D
:102A3800E18875F8D6B50D04E7F8F70065F8D6B55E
:102A48008AE60460E14875F8D6B50D04E7F8FB009E
:102A580065F8D6B58AE60570E7F8FD0065F8D6B5DD
:102A68000D03E12875F8D6B5E008CA001E2CE00869
:102A7800BB1CE038BB21E008CA00B82BE6FC1900F3
:102A8800E6F4CA2BCA004A38F0A4F0B5F09FF08EDD
:102A9800CA005C39F05FF04EF6FED0B5F6FFD2B54D
:0A2AA800DA004438FCFFFCFECB000E
:0E2AB200F04849813D021EE0CB001FE0CB0042
:102AC000F04809802D2629828D2E2D2829828D30CF
:102AD0002D5807F8F3002D1129812D0C07F8F2006D
:102AE0002D0F29828D132D0F07F812003D648FE200
:102AF0005FE6CB005FE68EE2CB008FE25EE6CB00C6
:102B00005FE26FE2CB006FE25EE2CB005FE26EE27B
:102B1000CB008FE25FE65FE26FE2CB005FE68EE222
:102B20006FE25EE2CB008FE25EE65FE26EE2CB0038
:102B30008AE60550E7F8F100F7F8D4B50D0B8AE204
:102B40000580E7F8F200F7F8D4B50D04E7F8F000D7
:102B5000F7F8D4B58AE20560E7F8F100F7F8D5B5E3
:102B60000D0B8AE20550E7F8F200F7F8D5B50D0431
:102B7000E7F8F000F7F8D5B55EE68EE26EE25EE2C9
:102B8000CB00F3FAD4B547FAF1003D038FE25EE6DD
:102B90000D0547FAF2003D025FE68EE2F3FAD5B585
:102BA00047FAF1003D035FE26EE2CB0047FAF20024
:082BB0003D026FE25EE2CB0082
:102BB800F04849813D033EE26EE6CB003FE26FE616
:022BC800CB0040
:102BCA002802D7000300F3F8FFFFB98087788787C8
:042BDA000802CB0022
:10350C00F2F408F1C0847C54E11C49863D01E10CC5
:10351C00F048F05926F4802538502D2426F4C0129A
:10352C0038502D2726F4C01238502D2A26F4802529
:10353C0038502D2D26F4802538502D3026F4004B94
:10354C0038502D3326F400E138502D3626F4C05077
:10355C0036F5FEFF3D36E6F5D70049C02D34E6F5CD
:10356C004F010D31E6F56B0049C02D2DE6F5A70096
:10357C000D2AE6F5470049C02D26E6F56F000D2310
:10358C00E6F5350049C02D1FE6F553000D1CE6F598
:10359C00230049C02D18E6F537000D15E6F51A0085
:1035AC0049C02D11E6F529000D0EE6F5110049C0B4
:1035BC002D0AE6F51B000D07E08549C02D04E0D56A
:1035CC000D02E128CB0076E2000476E3000466E30A
:1035DC00FFF7E6B68400E6B7040049C02D03E65BAE
:1035EC006F010D02E65B6201F6F5B4FEE6D81188B8
:0435FC00E108CB0017
:0E360000E6B60000E6B70000E6D80000CB00FA
:1037C400F68EE6B5F2F408F1C0847C5449863D05D2
:1037D400E6F4B70BF6F4E8B50D04E6F49711F6F445
:1037E400E8B5F224E8B5E6A48100E6B45C006FA471
:0437F400E108CB001D
:0637F800E6B40000CB0066
:0637FE00F2F4E6B5CB0079
:10380400E006E0070D08CC00CC00CC00CC00CC00D6
:10381400CC0008611870F046F057204830598DF3F9
:02382400CB00D7
:10382600C6030300CC00F6F020FCC60820FCCC0042
:0E383600F224E8B5248FE6B5FC08FC03FB88FD
:10399000D440F0B460FF000062FF000064FF00004C
:1039A00066FF000068FF00006AFF00006CFF000077
:1039B00070FF00009CF1000072FF000074FF000027
:1039C00076FF000094F100008CF1000084F100000B
:1039D00078F1000076F1000074F1000072F100004F
:1039E00070F100006EF100006CF100006AF100005F
:1039F00068F1000066F1000064F1000062F100006F
:103A000060F1000086FF000084FF000082FF0000DC
:103A100080FF00007EFF00007CFF00007AFF0000B6
:103A200078FF00009CFF00009EFF00007AF100007C
:103A30007CF1000098FF000088FF00008AFF000072
:103A40008CFF00008EFF000090FF000092FF00003E
:103A500094FF000096FF000086F100008EF1000048
:083A60009EF10000A8FF000028
:1036FC00ECFEECFFF0E8F0F9BB4AF6FEC4B5F6FFC1
:10370C00C6B55FE36FE38FE35FE75FE26FE28FE2E3
:10371C005FE6DFE3D180DEE39FE3D1809EE3DEE270
:10372C009EE26FE7D1806FE73FE3D1803FE36FE626
:10373C003FE27FE71FE1D1801FE17EE61FE0E10859
:06374C00FCFFFCFECB00B7
:06375200B748B7B7CB0039
:10375800D120BE88CC00CC00CA000036BB1AE6FCDB
:103768001900E6F4BA37CA004A38F0A4F0B5F2F8FE
:10377800C4B5F2F9C6B5CA005C39F2F4C4B5F2F5BD
:08378800C6B5DA004438CB009D
:0A379000E6D70100A758A7A7CB0059
:10379A00E10EE006C0E45C24D454F2B4D444F0B49C
:1037AA00CA007838B86409E147FE35008DF3CB00CA
:0A37BA00E60C0510FA000000CB0039
:10360E00C6030300CC00F6F040FCC60840FCCC001C
:06361E00FC08FC03FB8820
:10362400C6030300CC00F6F060FCC60860FCCC00C6
:10363400EC00C6871000EC06EC07F2F116B4D44196
:103644006E00F084CA00A403FC07FC06FC87FC009F
:06365400FC08FC03FB88EA
:10365A00C6030300CC00F6F040FCC60840FCCC00D0
:10366A00EC00C6871000EC06EC07F2F9ECB4F2F8AD
:10367A00EAB4CA00182AFC07FC06FC87FC00FC080E
:04368A00FC03FB88BA
:10368E00C6030300CC00F6F040FCC60840FCCC009C
:10369E00EC00C6871000EC06EC07CA00EC29FC070C
:0C36AE00FC06FC87FC00FC08FC03FB8809
:1036BA00C6030300CC00F6F060FCC60860FCCC0030
:1036CA00EC00C6871000EC06EC07CA005237FC076C
:0C36DA00FC06FC87FC00FC08FC03FB88DD
:1036E600C6030300CC00F6F080FCC60880FCCC00C4
:0636F600FC08FC03FB8848
:0A33980055534220737461636B000B
:063A68000240EEB4000074
:023A6E000083D3
:10201600ECFDECFEECFFF0DAE00E3E00E004F6F438
:10202600EEB4F04829812D0409813D041E000D03FC
:102036001F000D01E01EF04E49803D1DF04909804C
:102046002D1229813D172F00F04B704C2D05F6FB04
:10205600EAB4F6FCECB40D0FE004F6F4EAB4F6F4D8
:10206600ECB4E01E0D082E00E004F6F4EAB4F6F433
:10207600ECB40D01E01EF04E49803D12F2FF10FF58
:102086006688FFF7CA00FC23F6FF10FFCA00582433
:10209600CA007024CA004C23F04DC088CA007A02D8
:0A20A600F04EFCFFFCFEFCFDCB0039
:1020B000D1A066B7BFFF66BBBFFF66BCBFFFD1A0A4
:1020C00066B8BFFF66BABFFF66B9BFFF66C9BFFF8C
:1020D000E102C025F0455C3420455C2400455C14D9
:1020E000D47430B4D4642EB4DC07A8466EF4DC0794
:1020F000B846C025F0455C3420455C2400455C149E
:10210000D47440B4D4643EB4DC07A8466EF4DC0753
:10211000B846092149238DDDCA007024E018CA00A1
:042120007A02CB0074
:0A212400F2F116B4D4412400CB0000
:10212E00E11AF6F8EEB4F2F4EEB42D053F00D180CC
:0A213E0076B84000E10AF18ACB00F8
:10214800ECFF4A88FFB0D120BE88CC00CC00D180FB
:1021580066B8BFFFE004F6F4EEB43E004AFF880B11
:04216800FCFFCB00AD
:10216C00F04809803D1EE6F40001D7200000F6F48B
:10217C00F0F5F68EF2F5F78EF4F5E6F4ECF5E6F5FF
:10218C000000F6F4C8B4F6F5CAB4E6F6F6F5E6F7D0
:10219C000000F2F5CAB4F2F4C8B4DC15B864C47427
:0421AC000200CB0062
:1021B000E11CF2F216B4D4326E002D3CF048498096
:1021C0002D38F0736873C08440473D34F04949802E
:1021D0003D0AF04AC0855C25F0C366FC0C0040C592
:1021E0003D29E10C0D27F04949813D0AF04AC0859F
:1021F0005C45F0B366FB300040B53D1CE10C0D1AA8
:10220000F04949823D0AF04AC0855C65F01366F1E9
:10221000C00040153D0FE10C0D0DF04949833D0A0A
:10222000F04AC0855C8566F3000340353D03E10C50
:082230000D01E10CF18CCB0063
:0A223800F2F116B4D4416E00CB00A1
:10224200ECFDF028F039E6F400F9F0D4E6F99873E1
:10225200F08428810881E9893DFDE10AE4AD0A00A4
:10226200E12AE4AD0B00E10AE4AD0C00E10AE4ADC1
:102272000D00F05AE4AD0E00F04270432D11F04A09
:1022820047F81200ED0DC08CF0B3F0A2F04D06F449
:102292000F00CA004A38F084F095CA005C390D0D6F
:1022A200E6FB1200E00CE00AF04D06F40F00CA0053
:1022B2004A38F084F095CA001E39E108FCFDCB00D3
:1022C200ECFDECFEECFFF0DAF0E8F0F92802E6F4BF
:1022D20000F9B840E0AAE6F99873E6F800F9CA00F6
:1022E200F03848402D02E1180D2BA810F4810A00A5
:1022F2002D02E1180D25A810F4810B0049822D0250
:10230200E1180D1EA810F4810C004980FD02E118AD
:102312000D17F04E704F2D1348D02D11A810F4A1B7
:102322000E00B9ADA98DC08CA84006F40F00CA00FA
:102332004A38F0A4F0B5F09FF08ECA005C39E1088B
:0A2342000802FCFFFCFEFCFDCB00CE
:10234C00E6F50004F2F418B4C4545C00F2F418B4CA
:10235C00C4545E00F2F418B4C4546000F2F418B41F
:10236C00C4546200F2F418B4C4546400F2F418B407
:10237C00C4546600F2F418B4C4546800E005F2F4D6
:10238C0016B4C4543600F2F416B4C4543800F2F443
:10239C0016B4C4543E00F2F416B4C4544000F2F423
:1023AC0016B4C4544600F2F416B4C4544800F2F403
:1023BC0016B4C4544E00F2F416B4C4545000F2F4E3
:1023CC0016B4C4545600F2F416B4C4545800F2F4C3
:1023DC0016B4C4545E00F2F416B4C4546000F2F4A3
:1023EC0016B4C4546600F2F416B4C4546800CB009E
:1023FC00D1B0E60AF00EE68AAF04E60BE00EE68BEF
:10240C00AF04D1A0E60CD00EE68CAF04E6BD1B00E9
:10241C00E6C11A00E6CF2500E6C20000E6CE0000B9
:10242C00E6C32400D190E6BC1900E6BB21009A005B
:10243C000720D190E6BA2200E6B92300E6C92700AE
:0C244C00D190E6B83000E6B72600CB00C7
:10245800E6F400EEF6F416B4E6F400EDF6F418B47B
:08246800E005C4546C00CB0038
:10247000E10EE10CC0E5F0455C3420455C240045EC
:102480005C14E4C452B409E149E38DF4F2FA18B4DF
:10249000F04A06F43400CA004A38F6F442B4F6F5BD
:1024A00044B4F06A06F61000F046CA004A38F6F462
:1024B00046B4F6F548B4F07A06F75800F047CA007B
:1024C0004A38F6F422B4F6F524B4F2FB16B4F04B15
:1024D00006F43000CA004A38F6F426B4F6F528B4FB
:1024E000F06B06F62E00F046CA004A38F6F42AB41D
:1024F000F6F52CB4E6F482FFE005F6F42EB4F6F51A
:1025000030B4F08A06F83800F048CA004A38F6F4C9
:102510004AB4F6F54CB4F09A06F91400F049CA0032
:102520004A38F6F44EB4F6F550B406FA5A00F04ABA
:10253000CA004A38F6F432B4F6F534B4F07B06F744
:102540003400F047CA004A38F6F436B4F6F538B429
:1025500006FB3200F04BCA004A38F6F43AB4F6F5FE
:102560003CB4E6F47AF1E005F6F43EB4F6F540B496
:0E257000E008CA006C21E0F4F6F4E8B4CB00F9
:063A70000240D8B51AB4B3
:10257E00C6030300CC00F6F0A0FCC608A0FCCC00FD
:10258E00EC00C6871000EC06EC07F2F8D8B5D4586C
:10259E001E00D4481C00DC05A854F6F5DCB5FEF58B
:1025AE00F6F5DAB5F488380029862D6C098507F81A
:1025BE00F9FF9D0629822D1729822D15EA009E27E7
:1025CE00F2F4DCB58AF402F0EA009E27D4781A0001
:1025DE00D4681800DC07A846FEF4DC07B846CA002B
:1025EE00FC04EA009E27F2F4DCB58AF402F0EA005D
:1025FE009E27F2F4DAB53D42F2F1D8B5D4711A0045
:10260E00D4611800DC07A846FEF4DC07B846F2F7E2
:10261E00D8B5F487380047F80C003D05E1DAE4A799
:10262E003800EA009E27E6F60004D4570A00D44785
:10263E000800DC05B864E10AF2F4D8B5E4A4380069
:10264E00E006F2F5CAB4F2F4C8B4DC05C4640600C0
:10265E00F2F5CAB4F2F4C8B4F06406F60A00F075E6
:10266E00DC15B864C4740200E10CF2F5CAB4F2F4DD
:10267E00C8B4DC05E4C40800EA009E27CA00FC04C6
:10268E00EA009E27F2F4DCB59AF460F0F2F1D8B5C8
:10269E00D4711A00D4611800DC07A846FEF4DC07DA
:1026AE00B846F2F4DAB53D03CA00FC040D71F2F738
:1026BE00CAB4F2F6C8B4DC07D446060002F4DAB5A2
:1026CE00DC07C4460600F2F5D8B5D445060022F460
:1026DE00DAB5C4450600F2F6D8B5D44606003D1369
:1026EE00E19AE4A63800E009E008CA00061AF2F4FE
:1026FE00EAB53D4EE11CF2F5CAB4F2F4C8B4DC05FD
:10270E00E4C408000D45F2F7CAB4F2F6C8B4DC070B
:10271E00D48606000068F04606F40A00F057F0640E
:10272E00F2F1D8B5D4513200D4413000DC15B86482
:10273E00C4740200F2F1D8B5D4711A00D461180035
:10274E00DC07A846FFF4DC07B8460D22F2F7CAB440
:10275E00F2F6C8B4DC07D48606000068F04606F42C
:10276E000A00F057F064F2F1D8B5D4513200D441DA
:10277E003000DC15B864C4740200F2F1D8B5D4711F
:10278E001A00D4611800DC07A846FFF4DC07B8462F
:0E279E00FC07FC06FC87FC00FC08FC03FB8823
:063A76000240C8B51AB4BD
:063A7C000240CAB5000083
:063A82000240CCB500007B
:063A88000240CEB51AB4A5
:023A8E000084B2
:101A0600F2F7CEB5F4C73800F18C2986EA20901B90
:101A16002982EA20901B07F8080007F8F6FF9D02C6
:101A2600EA00901B49C03D03E12AE4A7380048902C
:101A3600FD78F2F616B4D45610009AF503000EF5AA
:101A4600C4561000F2F4CEB5C4940400E005F2F4D6
:101A5600CEB5C4540200F2F7CAB4F2F6C8B4DC1725
:101A6600D4560200A846F064F075F2F1CEB5D45112
:101A76002E00D4412C00DC15B864C4740200F2F6C2
:101A8600CEB5A8564095ED03E1CAE4A63800E006B7
:101A9600F2F1CEB5D4510A00D4410800DC05B86491
:101AA600F2F1CEB5D4510E00D4410C00DC05B86479
:101AB600F2F9CEB5D4590400A84940459D02A8596B
:101AC6000D02D4590400D4790A00D4690800DC0751
:101AD600A8467045DC07B846F2F1CEB5D4710A00C7
:101AE600D4610800DC07A846DFF4DC07B846F048F6
:101AF60049803D0BF2F1CEB5D4710A00D4610800DD
:101B0600DC07A846EFF4DC07B846F2F1CEB5D4718F
:101B16000A00D4610800DC07A846FFF4DC07B846D3
:101B26000D32F2F716B4D46714009AF60500686110
:101B3600F0567851C4571400E006F2F1CEB5D451F0
:101B46000A00D4410800DC05B864E6F60004F2F1A8
:101B5600CEB5D4510A00D4410800DC05B864E016BD
:101B6600F2F1CEB5D4510E00D4410C00DC05B864B8
:101B7600F2F1CEB5D4710A00D4610800DC07A8469C
:0E1B8600FFF4DC07B846E108CB00E118CB0005
:101B9400F048C089F0B95C3B20B95C2B00B95C1BF0
:101BA400D45B28B4D44B26B4DC05A8449AF4410091
:101BB400F48B52B447F809002D3CD47B30B4D46B79
:101BC4002EB4DC07A8466EF4DC07B846E6F700043A
:101BD400F048C085F0655C3620655C2600655C16BF
:101BE400D45624B4D44622B4DC05B874F048C08674
:101BF4005CC6F2F516B4D44510007046C445100016
:101C0400F2F516B4D4451000BFF4C4451000F048F2
:101C1400C085F0455C3420455C2400455C14D474D4
:101C240030B4D4642EB4DC07A8466FF4DC07B8469D
:101C3400CB00D47B30B4D46B2EB4DC07A8466EF44E
:101C4400DC07B846E6F70004F048C085F0655C366A
:101C540020655C2600655C16D45624B4D44622B4B0
:101C6400DC05B874F048C085F0455C3420455C243C
:101C740000455C14D47430B4D4642EB4DC07A84694
:081C84006FF4DC07B846CB0049
:101C8C00C6030300CC00F6F0A0FCC608A0FCCC00F8
:101C9C00EC00C6871000EC06EC07F2F116B4D44148
:101CAC001400F6F4CAB5F2FAC8B5F48A38002981E2
:101CBC00EA20601E29822D1229812D1029812D0EDA
:101CCC0029822D0C2982EA20BA1E29832D0729810D
:101CDC00EA20BA1E07F80B00EA300820F2F4CAB565
:101CEC008AF40200EA000A1EA85AD47A040040754D
:101CFC00FD05F0872085C48A04000D0840753D025F
:101D0C004F000D014E00E005C45A0400F2F5C8B5B1
:101D1C00D44502000841C4450200F2FBC8B5D44BBF
:101D2C0004004840FD50A85BD44B02001B45F2F860
:101D3C000EFEF2F7CAB4F2F6C8B4DC17D4560200A1
:101D4C00A8460048F064F075D45B2E00D44B2C00F0
:101D5C00DC15B864C4740200F2F1C8B5D4710A0081
:101D6C00D4610800DC07A84666F4007CDC07B846A2
:101D7C00F2F8C8B5D4780400A85840579D02A8487A
:101D8C000D02D4480400F6F4CCB54075ED03E1CA5D
:101D9C00E4A83800F2F1C8B5D4710A00D461080087
:101DAC00DC07A84672F4CCB5DC07B846F2F1C8B52E
:101DBC00D4710A00D4610800DC07A846FFF4DC07E4
:101DCC00B846EA0008209A000A40E19AE4AB3800D1
:101DDC00E009E008CA00061A4E00EA000820E1AA51
:101DEC00E4AB3800F2F1C8B5D4710A00D461080034
:101DFC00DC07A846FEF4DC07B846EA000820D47AD3
:101E0C000A00D46A0800DC07A84666F4007CDC07EC
:101E1C00B846F2F8C8B5D4580400A84840459D020D
:101E2C00A8580D02D4580400D4780A00D4680800CD
:101E3C00DC07A8467045DC07B846F2F1C8B5D4718A
:101E4C000A00D4610800DC07A846FFF4DC07B8469A
:101E5C00EA000820F2F5CAB4F2F4C8B4F06406F64D
:101E6C000A00F075DC15B864C4740200E006F2F5E3
:101E7C00CAB4F2F4C8B4DC05C4640600F2F4C8B504
:101E8C00C4640400E10AF2F4C8B5E4A43800F2F129
:101E9C00C8B5D4710A00D4610800DC07A846FEF46A
:101EAC00DC07B846E008CA00A403EA000820F2F4F4
:101EBC00CAB58AF40200EA00E01FF2F1C8B5D47189
:101ECC000A00D4610800DC07A846FEF4DC07B8461B
:101EDC00E006F2F1C8B5D4510A00D4410800DC0583
:101EEC00B864E6F60004F2F1C8B5D4510A00D44146
:101EFC000800DC05B864F2F1C8B5D4510E00D44129
:101F0C000C00DC05A8449AF40F00F2F516B4D44585
:101F1C00100066F4FF8FC4451000F2F516B4D445DA
:101F2C001000BFF4C4451000F2F1C8B5F4813800BC
:101F3C0047F80D003D1DE006F2F5CAB4F2F4C8B442
:101F4C00DC05C4640600F2F5CAB4F2F4C8B4F0645B
:101F5C0006F60A00F075DC15B864C4740200E10CD6
:101F6C00F2F5CAB4F2F4C8B4DC05E4C408000D2CD4
:101F7C00F2F9CAB4F2F8C8B4DC09F4280800492410
:101F8C003D11E11CDC09E4C80800F2F5CAB4F2F416
:101F9C00C8B4F06406F60A00F075DC15B864C474B5
:101FAC0002000D1249253D10E10CDC09E4C80800C3
:101FBC00F2F5CAB4F2F4C8B4F06406F60A00F0758F
:101FCC00DC15B864C4740200E10AF2F4C8B5E4A4E8
:101FDC0038000D14E016F2F1C8B5D4510E00D441FE
:101FEC000C00DC05B864F2F1C8B5D4710A00D461F8
:101FFC000800DC07A846FFF4DC07B846FC07FC0623
:0A200C00FC87FC00FC08FC03FB88C5
:102F0400ECFDECFFF0D94A88FFB0D120BE88CC009C
:102F1400CC00E008CA006C21E6FB0001E00CE00AEA
:102F2400F2F5CAB4F2F4C8B4DC15D4940200A8844F
:102F3400CA001E39F6FDEAB54AFF880BE108FCFF1A
:042F4400FCFDCB00C5
:102F4800F2F7CAB4F2F6C8B4DC07F4A6080049A13F
:102F58003D02E108CB0049A02D02E138CB00E12871
:022F6800CB009C
:102F6A00ECFF4A88FFB0D120BE88CC00CC00F2F931
:102F7A00CAB4F2F8C8B4DC09F488080049813D0FE4
:102F8A00E13CDC09E4C808004AFF880BF2F7CAB43E
:102F9A00F2F6C8B4DC17D4560200A8460D044AFF5C
:0A2FAA00880BE004E005FCFFCB00FB
:102FB400F2F3CAB4F2F2C8B4DC03F4820800498321
:102FC4003D1B48803D0CE006DC03C4620600F2F5BC
:102FD400CAB4F2F4C8B4DC05E4C408000D0BDC0385
:102FE400C4820600E12CF2F5CAB4F2F4C8B4DC05DC
:0C2FF400E4C40800E108CB00E118CB00A9
:103000001201000100000040D80802000001010286
:1030100000010000800000146080200024688040CF
:1030200000000000000000000000000000000000A0
:103030000000000000000000000000000000000090
:103040000000000000000000000000000000000080
:103050000000000000000000000000000000000070
:073060000000000000000069
:103068000403090400000000000000000000000044
:103078000000000000000000000000000000000048
:103088000000000000000000000000000000000038
:103098000000000000000000000000000000000028
:1030A8000000000000000000000000000000000018
:1030B8000000000000000000000000000000000008
:1030C80000000000000000000000000000000000F8
:1030D80000000000000000000000000000000000E8
:1030E80000002C03490058005800410054002000FB
:1030F8004100750074006F006D0061007400690084
:103108006F006E00200047006D006200480000005C
:1031180000000000000000000000000000000000A7
:103128000000000000000000000000000000000097
:103138000000000000000000000000000000000087
:103148000000000000000000000000000000000077
:103158000000000000000000000000000000000067
:103168000000000020035500530042002D004300DA
:1031780041004E00200043006F006D0070006100A8
:103188006300740000000000000000000000000060
:103198000000000000000000000000000000000027
:1031A8000000000000000000000000000000000017
:1031B8000000000000000000000000000000000007
:1031C80000000000000000000000000000000000F7
:1031D80000000000000000000000000000000000E7
:1031E80000000000000014035600300031002E00DB
:1031F800300030002E0030003000000000000000D9
:1032080000000000000000000000000000000000B6
:1032180000000000000000000000000000000000A6
:103228000000000000000000000000000000000096
:103238000000000000000000000000000000000086
:103248000000000000000000000000000000000076
:103258000000000000000000000000000000000066
:103268000000000000000000200343006600670023
:1032780020003100200049006600200030002000B6
:103288004100530020003100000000000000000051
:103298000000000000000000000000000000000026
:1032A8000000000000000000000000000000000016
:1032B8000000000000000000000000000000000006
:1032C80000000000000000000000000000000000F6
:1032D80000000000000000000000000000000000E6
:1032E80000000000000000000000090229000101A0
:1032F8000380C80904000000000000000904000160
:1033080002000000040705010240000007058202D0
:0333180040000072
:10027A00ECFDF04849813D5EF2F516B4D4457000B4
:10028A007841C4457000E00D86FD45008DFDF2F50C
:10029A0016B4D44570000EF4C4457000F2F516B4D5
:1002AA00D44510008FF4C4451000E6F5FF00F2F4BF
:1002BA0018B4C4546C00F2F516B4D4451000FFF417
:1002CA00C4451000E6F61230E6F70000F2F5CAB4AB
:1002DA00F2F4C8B4DC15B864C4740200E6F655003A
:1002EA00F2F5CAB4F2F4C8B4DC05C4640600E11835
:1002FA00F7F852B4F6F61AB4F2F62AB4F2F72CB4B6
:10030A00F2F544B4F2F442B4DC15B864C4740200E1
:10031A00F2F730B4F2F62EB4DC07A8466FF4DC0725
:10032A00B846F2F740B4F2F63EB4DC07A8466FF4DA
:10033A00DC07B846D1A076BB400076BC400076B751
:10034A0040009A001220D19076BA400076B9400057
:10035A0076C94000D1A066EDFFF376ED000466E0B1
:10036A00FFF2D18076E000080D07D19066BABFFF90
:10037A0066B9BFFF66C9BFFFF04849813D06E6F985
:10038A005500E008CA00061A0D06F2F116B4D4D1D7
:0A039A006E00F08DBB02FCFDCB00ED
:1003A400E009F2F4E8B446F40F00EA30D804F78E1A
:1003B40052B4E084F6F41AB4F2F62AB4F2F72CB488
:1003C400F2F544B4F2F442B4DC15B864C474020027
:1003D400E006F2F548B4F2F446B4DC15B894C4640B
:1003E4000200F2F730B4F2F62EB4DC07A8466FF43C
:1003F400DC07B846E006F2F524B4F2F422B4DC05D6
:10040400B864F2F724B4F2F622B4DC07A84676F412
:100414000030DC07B8469A000910F2F724B4F2F66B
:1004240022B4DC07A846EFF4DC07B846F2F63AB487
:10043400F2F73CB4F2F550B4F2F44EB4DC15B864FF
:10044400C4740200F2F740B4F2F63EB4DC07A846E6
:100454006FF4DC07B846F2F5CAB4F2F4C8B406F493
:100464000A00F064F075F2F54CB4F2F44AB4DC1509
:10047400B864C4740200E6F6FF03F2F534B4F2F48F
:1004840032B4DC05B864F2F734B4F2F632B4DC0703
:10049400A846BFF4DC07B846F2F734B4F2F632B437
:1004A400DC07A84676F40030DC07B8469A00091049
:1004B400F2F734B4F2F632B4DC07A846EFF4DC0702
:1004C400B846F2F734B4F2F632B4DC07A846FEF4C8
:1004D400DC07B84642F8E8B42D0C48802D0AC2F473
:1004E4000770F6F41AB4F09868937C28F6F9E8B427
:0804F400CB00F6F8E8B4CB00E0
:1004FC00F2F730B4F2F62EB4DC07A8466EF4DC0743
:10050C00B846F2F730B4F2F62EB4DC07A8467EF407
:10051C00DC07B846F2F740B4F2F63EB4DC07A84666
:10052C006EF4DC07B846F2F740B4F2F63EB4DC07E2
:10053C00A8467EF4DC07B846F2F724B4F2F622B4EF
:10054C00DC07A846FEF4DC07B846F2F734B4F2F642
:10055C0032B4DC07A846FEF4DC07B846E6F6000425
:10056C00F2F524B4F2F422B4DC05B864F2F534B438
:10057C00F2F432B4DC05B864F2F516B4D4451000CC
:10058C0066F4FF8FC4451000F2F516B4D445100084
:10059C00BFF4C4451000E006F2F5CAB4F2F4C8B4D6
:1005AC00DC05C4640600F2F5CAB4F2F4C8B4F06415
:1005BC0006F60A00F075DC15B864C4740200E10C90
:1005CC00F2F5CAB4F2F4C8B4DC05E4C40800F78E42
:1005DC0052B4E6FB0001E00CE00AF2F5CAB4F2F406
:1005EC00C8B4DC15D4940200A884CA001E39F2F7F2
:1005FC00CAB4F2F6C8B4DC07D48606000068F0462C
:10060C0006F40A00F057F064F2F54CB4F2F44AB474
:10061C00DC15B864C4740200F2F738B4F2F636B4E0
:10062C00DC07A846FEF4DC07B846F2F734B4F2F661
:10063C0032B4DC07A846FFF4DC07B846F2F730B456
:10064C00F2F62EB4DC07A8466FF4DC07B846F2F7D6
:10065C0040B4F2F63EB4DC07A8466FF4DC07B846AB
:02066C00CB00C1
:10066E00C6030300CC00F6F0A0FCC608A0FCCC002C
:10067E00EC00C6871000EC06EC0706F0F8FFF2F16E
:10068E0016B4D4412600B980F2F116B4D441260036
:10069E007C84E4800100F2F116B4D4412800C440F9
:1006AE000200F2F116B4D4412A00C4400400F2F163
:1006BE0016B4D4412C00C4400600F2F5CAB4F2F4CC
:1006CE00C8B4DC05F484080049833D09E198F7F8C5
:1006DE0052B4E009E008CA00061AEA003E09A980F1
:1006EE0067F84000C08406F4C0FF2D0E06F44000EB
:1006FE00EA303E09F48001002986EA303E09F08096
:10070E00CA005009EA003E09A9808AF40270EA0084
:10071E001E08F2F4EAB52D33F2F7CAB4F2F6C8B4F5
:10072E0006F60A00F2F5CAB4F2F4C8B4DC07B864EF
:10073E00DC05C4740200E086F2F5CAB4F2F4C8B463
:10074E00DC05C4640600E08CF0A0E00B06FA004065
:10075E0016FB0000F2F5CAB4F2F4C8B4DC15D4945A
:10076E000200A884CA005C39E11CF2F5CAB4F2F4A6
:10077E00C8B4DC05E4C40800F2F4EAB5AB04F2F93F
:10078E00CAB4F2F8C8B4DC09F4A8080049A22D02D4
:10079E0049A43D35E14CDC09E4C80800E178F7F8DE
:1007AE0052B48A001610F2F7CAB4F2F6C8B4DC07D7
:1007BE00D4460600D45006004054FD04DC07D496FF
:1007CE0006000D02D4900600E018CA00061AEA00D0
:1007DE003E09F2F7CAB4F2F6C8B4DC07D4460600F6
:1007EE00D45006004054FD04DC07D49606000D02DA
:1007FE00D4900600E008CA00061AEA003E09E19805
:10080E00F7F852B4E009E008CA00061AEA003E09F9
:10081E00F2F5CAB4F2F4C8B4DC05F48408002D2D48
:10082E00E006F2F4C8B4DC05C4640600F2F5CAB4FE
:10083E00F2F4C8B4F06406F60A00F075DC15B8647C
:10084E00C4740200E6FB0001E00CE00AF2F5CAB443
:10085E00F2F4C8B4DC15D4940200A884CA001E3980
:10086E00E10CF2F5CAB4F2F4C8B4DC05E4C4080035
:10087E00F78E52B4E008CA00941BF2F7CAB4F2F62F
:10088E00C8B4DC07F48608003D4CE08CF0A0E00B09
:10089E0006FA004016FB0000DC17D4960200A8866C
:1008AE00CA005C39E086F2F5CAB4F2F4C8B4DC05CD
:1008BE00C4640600E14CF2F5CAB4F2F4C8B4DC0527
:1008CE00E4C40800D45006004850FD23F6F520B4C9
:1008DE00E168F7F852B4F2F7CAB4F2F6C8B4DC170E
:1008EE00D4560200A84606F40800F064F075F2F53E
:1008FE004CB4F2F44AB4DC15B864C4740200F2F7D6
:10090E0034B4F2F632B4DC07A846FFF4DC07B8467E
:10091E000D0FE198F7F852B4E009E008CA00061A84
:10092E000D07E198F7F852B4E009E008CA00061A7C
:10093E0006F00800FC07FC06FC87FC00FC08FC0324
:02094E00FB8824
:10095000ECFDECFEF0D82804E6F4F232E6F50000F7
:10096000B840C4500200F2F9CAB4F2F8C8B4DC09C5
:10097000F48808002D04E10CDC09E4C80800D44D1B
:1009800002007C8429822D3E2981EA20A00A098266
:10099000EA30420BD45D0600C2F400704045FD030E
:1009A000D4ED06000D02C2FE0070C2F40770F6F42A
:1009B0001AB4E138F7F852B4F2F5CAB4F2F4C8B494
:1009C000DC05C4E40600F0CEE6FA0030E6FB0000E9
:1009D000F2F9CAB4F2F8C8B406F80A00CA005C39E1
:1009E000F2F5CAB4F2F4C8B4F06406F60A00F07581
:1009F000DC15B864C4740200F09EE018CA00061A40
:100A0000EA00440BD44D02004981FD0AE198F7F851
:100A100052B4E009E008CA00061AE118EA00440BE3
:100A2000D4900200A880DC09F4880300C0865C86AC
:100A3000DC09F4880200C084F0E470E6D45D0600AE
:100A400040E5FD03D4ED06000D00C2F40770F6F496
:100A50001AB4E148F7F852B4F2F5CAB4F2F4C8B4E3
:100A6000DC05C4E40600F0CED4B00200A8A0F2F980
:100A7000CAB4F2F8C8B406F80A00CA005C39F2F544
:100A8000CAB4F2F4C8B4F06406F60A00F075DC15D6
:100A9000B864C4740200F09EE018CA00061A0D5231
:100AA000D44D02004984FD09E198F7F852B4E009F9
:100AB000E008CA00061AE1180D45D45D020066F58B
:100AC000FF00F0455C6500545C15E6F46870004575
:100AD000CA004A38F064F075DC05A924C025D44D5D
:100AE000060040459D03D4ED06000D01C02EC2F462
:100AF0000770F6F41AB4E158F7F852B4F2F5CAB434
:100B0000F2F4C8B4DC05C4E40600F0CEF0B7F0A6F9
:100B1000F2F9CAB4F2F8C8B406F80A00CA005C399F
:100B2000F2F5CAB4F2F4C8B4F06406F60A00F0753F
:100B3000DC15B864C4740200F09EE018CA00061AFE
:0C0B40000D01E1180804FCFEFCFDCB00D8
:06384400ECF5ECF4DB00E2
:10384A00AAF408F0AAF403E0F2F500FE0D0AF2F574
:10385A0002FE0D07AAF403E0F2F504FE0D02F2F5EA
:0E386A0006FE4AF5F40E4AF5F41F7C25CB004D
:1038780000441055004410557C2442F506FE2D0FD7
:1038880042F502FE2D0942F504FE2D0366F4FF3FC2
:10389800CB00FFF4EEF4CB00EFF4FEF4CB0076F4AB
:0438A80000C0CB0091
:1038AC00DC459964DC07B966086128213DF9E6031B
:0438BC000300CB003A
:10393E00F01999882D03498D2DFC28112989D084E1
:0E394E002D028D02E014CB00E6F4FFFFCB004B
:0C397200F04828810881E9893DFDCB0068
:1038F0000D09A9882D0328A148A03D02E004CB00B2
:1039000008810891A9A9A988418A2DF3A9A9A988A4
:0E391000418AFD02E014CB00E6F4FFFFCB007D
:10395C00F0480D05DC0B99AADC09B9A80881A00C6C
:06396C003DF9F059CB000B
:1038C00088C0A860D4700200F028F0390D0ADC0B23
:1038D000A98ADC03B9820821183008A118B0286130
:1038E0003870F04670473DF3F048F0590802CB00BD
:10391E00F028F0390D0728B138C0F06ADC09B9C8B3
:10392E0008811890F04B704C3DF6F042F053CB00EE
:023A9000000034
:04009C000040D7B594
:0400A0000340DEB586
:0400A4000100000057
:0400A8000340E2B57A
:0400AC000640D0B585
:0400B0000340E6B56E
:0400B400D740F0B48D
:0400B800D94016B461
:0600BC000D810300ECF5CC
:0400C2000300010036
:0400C6000540D8B564
:0400CA000740C8B56E
:0400CE000100040029
:0400D2000140EAB54A
:0200D600000028
:04000000FA00000101
:04000800FA00D433F3
:04001000FA001434AA
:04001800FA00543462
:04002800FA00943412
:04005400FA008C1C06
:04007400FA00BA369E
:04009800FA0026380C
:0400DC00FA002436CC
:0400E000FA00E63606
:0400E400FA008E365A
:0400E800FA005A368A
:0400EC00FA000E36D2
:0400F000FA006E069E
:0400F400FA007E256B
:00000001FF
